:020000020000FC
:020000000FC02F
:0200060073C0C5
:100020000FE90DBF0DE007BB02E008BB00E004BB19
:1000300000E00FBD05E003BF02E009BF789400E0D7
:10004000009364000FD000916400003019F4C09A4E
:10005000C39AF8CF013009F4F5CF023011F4C098FB
:10006000C398F0CFF89400270093620000936300D8
:10007000789406B3027049F0C2980091620004308F
:10008000C0F30027009364000895C29AF8940027F3
:100090000093620000936300789406B3027081F4C9
:1000A00000916200013020F4009163000C3FA8F33E
:1000B00006B30270E9F3C29802E000936400089569
:1000C000C29800916300023118F001E000936400CF
:1000D00008950EE10F9300E00F9300E00A95F1F709
:1000E0000F910A95C9F70F910A95A1F708950F93FB
:1000F0000FB70F931F932F931091630013951093D5
:10010000630029F4109162001395109362002F91FF
:0A0110001F910F910FBF0F9118957A
:00000001FF
